S02B00002F686F6D652F74696D652F646F632F636F646566696C652F656D62652F426C6F672F73746D33322FBD
S315080000000000022055170008511700084F1700086E
S315080000104F1700084F1700084F1700080000000088
S315080000200000000000000000000000005117000852
S315080000305117000800000000511700088D04000839
S315080000404F1700084F1700084F1700084F170008EA
S315080000504F1700084F1700084F1700084F170008DA
S315080000604F1700084F1700084F1700084F170008CA
S315080000704F1700084F1700084F1700084F170008BA
S315080002904F1700084F17000880B500AF41F6044015
S315080002A001F048FA082300220121104800F0F7FF60
S315080002B00823002200210D4801F011F808210B48F7
S315080002C000F0DEFF0A4B1B68094A43F4807313608B
S315080002D041F6024001F02EFA4FF4005302220021A3
S315080002E0044800F0DCFF00BF80BD00BF00100258C4
S315080002F0004802580008025880B500AF4FF4407015
S3150800030001F09BFA00F00EF84FF47A7000F09EF8B0
S31508000310FFF7C2FF00F026F900F03AF9052000F0D1
S315080003207BF8F9E780B58CB000AF3B462C2200215C
S31508000330184601F0A9FB41F6074001F0FBF941F622
S31508000340816001F0F7F9022301220121304800F00B
S31508000350A6FF0223022200212D4800F0C0FF002339
S31508000360FB6203E000BFFB6A0133FB62FB6A132BE7
S31508000370F8D90221264800F081FF00233B700223AA
S315080003807B70244B7B6005233B72C0237B81022351
S315080003903B7302237B730223BB7320233B748123A5
S315080003A07B8202233B7502237B750223BB752023C0
S315080003B03B7681237B8302233B7702237B770223C9
S315080003C0BB77002387F82030082387F821300423D9
S315080003D087F82230042387F82330042387F824304B
S315080003E0042387F82530042387F82630012387F865
S315080003F02730022387F82830002387F829303B4620
S31508000400184601F04DF800BF3037BD4680BD00BF25
S31508000410001C025840787D0180B485B000AF786032
S31508000420094B1B68FB6001E030BF00BF064B1A682A
S31508000430FB68D31A7A689A42F6D800BF00BF143709
S31508000440BD465DF8047B70474000002080B582B049
S3150800045000AF7860042001F0D3F9002001F02CF9F0
S3150800046002467B68B2FBF3F3013B184601F0C2F97A
S3150800047001F0DEF90F21FF2001F0E8F901F0CAF9D1
S3150800048001F0CFF900BF0837BD4680BD80B400AF84
S31508000490044B1B680133034A136000BFBD465DF871
S315080004A0047B70474000002080B582B000AF7860BA
S315080004B07B681B88002B0CD14FF40051074800F0CD
S315080004C0E2FE0346B3F5005F0CBF01230023DBB24F
S315080004D000E0002318460837BD4680BD00080258CC
S315080004E080B582B000AF78600B46FB70FB78032BB3
S315080004F020D801A252F823F0350500083505000872
S3150800050009050008230500087B68DB8A022B13D13E
S315080005107B681B88002B0FD108210B4800F0B6FE1C
S315080005200AE07B681B88002B08D10821064800F0E2
S31508000530ADFE03E000BF02E000BF00E000BF00BF61
S315080005400837BD4680BD00BF0010025880B400AF12
S31508000550034B1B681846BD465DF8047B704700BF11
S315080005604000002080B582B002AF064B0193064BCF
S315080005700093002300220121044800F0D3FA00BFAB
S31508000580BD4680BDE1040008A9040008000000205B
S3150800059080B500AFFFF7DAFF0346184600F032FCD5
S315080005A000BF80BD80B483B000AF78607B685B080D
S315080005B003F055337A68D31A7B607B6803F03332CD
S315080005C07B689B0803F0333313447B607B681A0906
S315080005D07B68134403F00F337B607A6813461B026B
S315080005E013441A0413441B0E18460C37BD465DF80F
S315080005F0047B704780B485B000AF786039603B688B
S315080006005B099B007A6813441B68FB603B6803F030
S315080006101F03FA6822FA03F303F001031846143796
S31508000620BD465DF8047B704780B485B000AF78603E
S3150800063039603B6803F01F03012202FA03F3FB60EB
S315080006403B685B099A0079680A441168FA68D243DC
S315080006509B00786803440A401A6000BF1437BD46F9
S315080006605DF8047B704780B485B000AF7860396068
S315080006703B6803F01F03012202FA03F3FB603B68A1
S315080006805B099A0079680A4411689B007A681344E2
S31508000690FA680A431A6000BF1437BD465DF8047B42
S315080006A0704780B487B000AFF860B9607A60BB68FD
S315080006B003F01F03012202FA03F37B617B68002B18
S315080006C00CD0BB685B099A00F9680A4411689B005C
S315080006D0FA6813447A690A431A600CE0BB685B0936
S315080006E09A00F9680A4411687A69D2439B00F86847
S315080006F003440A401A6000BF1C37BD465DF8047BF8
S31508000700704780B584B000AF786039600023BB605D
S315080007100023FB6015E0FB689B007A6813441B689E
S31508000720002B0BD0FB689B007A6813441B6818469D
S31508000730FFF738FF0246BB681344BB60FB6801330A
S31508000740FB603B68013B5B095A1CFB689A42E2D88E
S31508000750BB6818461037BD4680BD80B487B000AF69
S31508000760F860B9607A6000237B610CE07B699B00C6
S31508000770BA681A447B699B00F9680B4412681A60C8
S315080007807B6901337B617B68013B5B095A1C7B698A
S315080007909A42EBD800BF00BF1C37BD465DF8047B04
S315080007A0704780B487B000AFF860B9607A603B6084
S315080007B000237B6112E07B699B00BA6813441968C1
S315080007C07B699B007A6813441A687B699B00F86802
S315080007D003440A401A607B6901337B613B68013B2D
S315080007E05B095A1C7B699A42E5D800BF00BF1C37D3
S315080007F0BD465DF8047B704780B584B000AFF860ED
S31508000800B9607A607B68013B5B0901339B001A4635
S31508000810B968F86801F00AF9034618461037BD4664
S3150800082080BD80B483B000AF786039607A683B6871
S31508000830D31A18460C37BD465DF8047B704780B559
S3150800084086B000AFF8607B600B46FB721346BB723E
S315080008507D4B7B61FB689B69002B00F05F81BA7A50
S31508000860FB7A9A420CD0FB687A689A60BB7A002BAE
S3150800087006D0FB689B7843F00203DAB2FB689A70ED
S31508000880BB7A002B00F09880FB689B7803F0010385
S31508000890002B5FD1FB689B6819467868FFF7C1FF94
S315080008A00246FB689B691B889A42C0F23881FB683E
S315080008B0DB8A002B19D0FB681B6919467868FFF795
S315080008C0B0FF0246FB689B691B899A420DDBFB68F1
S315080008D0DB7803F00403002B04D07B699B690221B3
S315080008E0F8689847FB680022DA82FB687A68DA605B
S315080008F0FB6800229A82FB689B7843F00103DAB210
S31508000900FB689A70FB68DB7803F00103002B04D0C0
S315080009107B699B690021F8689847FB687A685A6082
S31508000920FDE0FB68DB68FA68926952891A44FB683D
S31508000930DA60FB689B8A01339AB2FB689A82FB6885
S31508000940DB7803F00803002B04D07B699B6903213D
S31508000950F8689847FB689B695B89002B0BD0FB6896
S31508000960DB6819467868FFF75CFF0246FB689B69F7
S315080009705B899A42D5DAFB68DB8A002B00F0CF80C8
S31508000980FB685B6819467868FFF74BFF0246FB6809
S315080009909B69DB889A4240F3C280FB68DB7803F0E8
S315080009A00403002B04D07B699B690221F8689847E9
S315080009B0FB680022DA82B2E0FB689B7803F0010349
S315080009C0002B7ED0FB689B6819467868FFF729FFDD
S315080009D00246FB689B695B889A42C0F2A080FB6866
S315080009E09B7823F00103DAB2FB689A70FB68DB7820
S315080009F003F00203002B04D07B699B690121F86888
S31508000A009847FB685B6819467868FFF70AFF02464D
S31508000A10FB689B699B889A4218DBFB685B681946EA
S31508000A207868FFF7FEFE0246FB689B69DB889A42F8
S31508000A300CDCFB68DB8A01339AB2FB68DA82FB6856
S31508000A407A681A6120E000BF44000020FB68DB8A50
S31508000A50002B16D0FB685B6819467868FFF7E1FE3D
S31508000A600246FB689B699B889A420ADAFB68DB7830
S31508000A7003F00403002B04D07B699B690221F86804
S31508000A809847FB680022DA82FB68DB8A002B14D0C1
S31508000A90FB68DA8AFB689B699B899A420DD1FB68D9
S31508000AA0DB7803F00403002B04D07B699B690221E1
S31508000AB0F8689847FB680022DA82FB687A685A6009
S31508000AC02DE0FB68DB8A002B1AD0FB681B691946E8
S31508000AD07868FFF7A6FE0246FB689B691B899A425F
S31508000AE01DDBFB68DB7803F00403002B04D07B696D
S31508000AF09B690221F8689847FB680022DA820EE0B3
S31508000B00FB689B7803F00203002B08D0FB689B78F0
S31508000B1023F00203DAB2FB689A7000E000BF1837C8
S31508000B20BD4680BD80B586B000AFF8607A601A46CB
S31508000B300B467B8113463B81124B7B617B6A002BFC
S31508000B4002D03B6A002B01D1002317E0282200219E
S31508000B50786900F099FF7B69FA681A607B697A8977
S31508000B609A807B697A689A607B693A899A817B69F7
S31508000B707A6A9A617B693A6ADA61012318461837F4
S31508000B80BD4680BD4400002080B586B000AF7860C1
S31508000B90224BFB6000233B6116E0FB68D969FB68C2
S31508000BA018683A691346DB009B1A9B0003441846EB
S31508000BB088470346BB72BB7A1A4639697868FFF7D5
S31508000BC070FD3B6901333B61FB689B881A463B69AC
S31508000BD09342E2DBFB681B697B61FB689B883B6190
S31508000BE013E0FB68DB697A690432104698470346C6
S31508000BF0FB72FB7A1A4639697868FFF752FD7B69FA
S31508000C001B687B613B6901333B617B69002BE8D13B
S31508000C1000BF00BF1837BD4680BD00BF4400002096
S31508000C2090B585B000AFF860B9607A603B60396806
S31508000C30B868FFF7DFFC0346DCB239687868FFF767
S31508000C40D9FC0346DAB23B6A2146F868FFF7F7FD96
S31508000C5000BF1437BD4690BD80B588B000AFF860B8
S31508000C60B9607A603B6007F1140300221A605A6083
S31508000C7040213868FFF745FD0346002B30D007F1C1
S31508000C80140040233A687968FFF78BFD07F11403CF
S31508000C90402239681846FFF7AFFD0346002B0CBF04
S31508000CA001230023DBB2FB7707F1140040233A68DF
S31508000CB0B968FFF776FD07F114034022396818462C
S31508000CC0FFF79AFD0346002B0CBF01230023DBB276
S31508000CD0BB77FA7FB97FBB6AF868FFF7B0FD00E01B
S31508000CE000BF2037BD4680BD90B589B002AF786099
S31508000CF03960434BBB600023FB6013E0BB6819688F
S31508000D00FA681346DB009B1A9B00C818BB6803F1F8
S31508000D1020013B680093FB687A68FFF781FFFB6850
S31508000D200133FB60BB689B881A46FB689342E5DB88
S31508000D30BB681B697B61BB689B88FB6010E07B69AD
S31508000D40181DBB6803F120013B680093FB687A68AD
S31508000D50FFF766FF7B691B687B61FB680133FB60F5
S31508000D607B69002BEBD10023FB601FE0BB68996809
S31508000D70FA681346DB0013449B000B4403F1080092
S31508000D80BB6803F12004BB689968FA681346DB0060
S31508000D9013449B000B441A463B68009313467A6833
S31508000DA02146FFF759FFFB680133FB60BB689B8947
S31508000DB01A46FB689342D9DBBB685B693B6110E066
S31508000DC03B6903F10C00BB6803F120013B691A1D5E
S31508000DD03B68009313467A68FFF73EFF3B691B683A
S31508000DE03B613B69002BEBD1BB6820334022796815
S31508000DF01846FFF7B2FC00BF1C37BD4690BD00BFC2
S31508000E004400002080B584B000AF786007F108037D
S31508000E1000221A605A6007F108031846FFF7B4FE65
S31508000E2007F1080379681846FFF75EFF00BF103719
S31508000E30BD4680BD80B485B000AF0F4B7B600023F4
S31508000E40FB607B681B69BB607B689B881A46FB68EE
S31508000E501344FB6005E0FB680133FB60BB681B6855
S31508000E60BB60BB68002BF6D1FB6818461437BD4635
S31508000E705DF8047B704700BF4400002080B487B04B
S31508000E8000AF0346FB801E4BFB6000237B610023FB
S31508000E907B6110E0FB6819687A691346DB009B1AC8
S31508000EA09B000B441B88FA889A4201D17B6921E092
S31508000EB07B6901337B61FB689B881A467B69934291
S31508000EC0E8DBFB681B693B61FB689B887B610CE080
S31508000ED03B699B88FA889A4201D17B690AE03B699B
S31508000EE01B683B617B6901337B613B69002BEFD152
S31508000EF04FF0FF3318461C37BD465DF8047B704734
S31508000F004400002080B487B000AF0346FB80224B24
S31508000F10FB6000237B6100237B6117E0FB6819688F
S31508000F207A691346DB009B1A9B000B441B88FA88D8
S31508000F309A4208D1FB6819687A691346DB009B1A3E
S31508000F409B000B4421E07B6901337B61FB689B882E
S31508000F501A467B699342E1DBFB681B693B61FB68C8
S31508000F609B887B610DE03B699B88FA889A4202D18F
S31508000F703B69043309E03B691B683B617B690133C4
S31508000F807B613B69002BEED1002318461C37BD4612
S31508000F905DF8047B704700BF4400002080B582B02E
S31508000FA000AF78607B681B881846FFF767FF034623
S31508000FB018460837BD4680BD80B582B000AF786058
S31508000FC07B689B881846FFF759FF0346184608377B
S31508000FD0BD4680BD80B582B000AF786039607B6859
S31508000FE039681846FFF73FFB00BF0837BD4680BD86
S31508000FF080B582B000AF786039607B68396818467A
S31508001000FFF712FB00BF0837BD4680BD80B584B028
S3150800101000AF78600B467B807B881846FFF72EFF6B
S31508001020F860FB68002B04DBF9687868FFF7D2FFE5
S3150800103000E000BF1037BD4680BD80B584B000AF64
S3150800104078600B467B807B881846FFF717FFF860A9
S31508001050FB68002B04DBF9687868FFF7C9FF00E036
S3150800106000BF1037BD4680BD80B483B000AF78603E
S315080010707B68002B07D07B689B7803F00103002B65
S3150800108001D0012300E0002318460C37BD465DF861
S31508001090047B704780B483B000AF78607B68002B10
S315080010A007D07B689B7803F00203002B01D001234D
S315080010B000E0002318460C37BD465DF8047B7047F0
S315080010C080B584B000AF374B3B6000237B6012E0ED
S315080010D03B6819687A681346DB009B1A9B000B4429
S315080010E01846FFF7D7FF0346002B01D0012354E02B
S315080010F07B6801337B603B689B881A467B68934212
S31508001100E6DB3B681B69FB603B689B887B600FE0FE
S31508001110FB6804331846FFF7BDFF0346002B01D0D2
S3150800112001233AE0FB681B68FB607B6801337B6040
S31508001130FB68002BECD100237B6013E03B689968C1
S315080011407A681346DB0013449B000B4408331846A1
S31508001150FFF7A0FF0346002B01D001231DE07B68A3
S3150800116001337B603B689B891A467B689342E5DBC3
S315080011703B685B69BB600CE0BB680C331846FFF73D
S3150800118089FF0346002B01D0012306E0BB681B68D4
S31508001190BB60BB68002BEFD1002318461037BD464D
S315080011A080BD00BF4400002080B586B000AF7860DF
S315080011B0184BFB60FB681B697B6100233B617B68FE
S315080011C0002B01D1002320E0FFF734FE03463F2B16
S315080011D001DD002319E07B69002B0FD1FB687A68D3
S315080011E01A61012311E07A697B689A4201D10023CA
S315080011F00BE07B693B617B691B687B617B69002B24
S31508001200F1D13B697A681A60012318461837BD463A
S3150800121080BD00BF4400002080B487B000AF78606E
S31508001220154BFB60FB685B697B6100233B617B6850
S31508001230002B01D1002319E07B69002B0FD1FB6835
S315080012407A685A61012311E07A697B689A4201D16A
S3150800125000230BE07B693B617B691B687B617B69CB
S31508001260002BF1D13B697A681A60012318461C37AE
S31508001270BD465DF8047B70474400002081617047D5
S31508001280090481617047006908407047436901EAAB
S31508001290030221EA030141EA0241816170472DE90F
S315080012A0F04105680026C4684FF0030E43FA06F7B6
S315080012B0FF070DD577000EFA07FC01FA07F802FAC0
S315080012C007F725EA0C0524EA0C0448EA05053C4319
S315080012D00136102EEAD10560C460BDE8F081012907
S315080012E041680CBF19439943F0B5416000248168F1
S315080012F0032643FA04F5ED0707D5650006FA05F750
S3150800130002FA05F521EA070129430134102CF0D128
S315080013108160F0BD2DE9F04391F800C0BCF1000FE3
S3150800132000F0A580012A26D0574B9E1F022A18BF17
S315080013301E46013A554D0023B1F8028045F8323071
S3150800134008F1FF3355F832402343D4B245F832301A
S31508001350A700B0FBFCF34E48FFB2B3FBF0FCACF1C0
S31508001360030001284B4808D80423D0F82CE4BB40D6
S315080013704EEA03030DE0484EDBE7ACF1050EBEF17D
S31508001380030F76D80823D0F82C9403FA07FE4EEA02
S315080013900903C0F82C340CFB08F3B3F5D27F09D83F
S315080013A0DFF8F0C00220DCF82CE4B84040EA0E0072
S315080013B0CCF82C046700087904EB4404E4B2B0B115
S315080013C055F832C000F1FF3E4CEA4E2CDFF8C4E077
S315080013D045F832C04FF4803CDEF82C840CFA04FC45
S315080013E0B3FBF0F04CEA080CCEF82CC430804879F0
S315080013F0B0B155F832C000F1FF3E4CEA0E4CDFF8AA
S3150800140094E045F832C04FF4003CDEF82C840CFA20
S3150800141004FCB3FBF0F04CEA080CCEF82CC4708040
S31508001420897999B155F8320001F1FF3C40EA0C6020
S3150800143045F832004FF480221648A240D0F82C54C2
S31508001440B3FBF1F32A43C0F82C24B380114AFFB248
S315080014504FF08073D2F80014BB400B43C2F8003437
S315080014604FF00073BB40D2F800141942FBD0BDE818
S31508001470F083DFF828E073458DD94FF00C0ED0F8CD
S315080014802C340EFA07FE73E7360000203044025863
S3150800149040420F00004002582A0000203F548900AD
S315080014A0F8B5814B0446D3F8002442F00102C3F88C
S315080014B00024D3F8102422F00702C3F81024D3F826
S315080014C0102412F0380FFAD10122C3F8002494F838
S315080014D0291094F8280000F02FFA94F8270000F055
S315080014E057FA94F8260000F0D3F994F82630002B22
S315080014F000F0C58000F0BCF963688BB16A4BD3F87D
S31508001500002442F48032C3F80024D3F8002492035E
S31508001510FBD563684FF47A72B3FBF2F3634A13841C
S31508001520237C227A1B03617843EA0213227E0B434B
S3150800153043EA02535C4AC2F82834002900F0A28024
S315080015406568002304F108012846C2F82C340122F4
S31508001550FFF7E0FE022204F110012846FFF7DAFE43
S315080015602846032204F11801FFF7D4FE23784F48D2
S31508001570002B40F08980C38994F8245000264A4FEE
S3150800158094F8201094F8212003800729C7F81864D6
S315080015904FEA0516D7F818C446EA012646EA0206AF
S315080015A046EA0C06C7F8186406D90B2994BF07390A
S315080015B0063943FA01F18BB2072A438009D90B2A67
S315080015C095BF073A911F43FA02F20B4194BF93B2B3
S315080015D09BB2032D94F82310334E8CBFEA1E1A468D
S315080015E04FF00005838084BF43FA02F292B20329C2
S315080015F0428194F82220C6F81C544FEA01258CBF74
S315080016000339194645EA0215D6F81C7488BF43FA09
S3150800161001F145EA070588BF89B2032AC6F81C54B2
S315080016208CBF033A1A46018188BF43FA02F294F83E
S31508001630251088BF92B20329C2801B4AD2F82044DB
S315080016404FF00004C2F82044D2F8204444EA0114BA
S3150800165084BF033943FA01F1C2F8204488BF8BB22C
S315080016608381D2F8103443F00303C2F81034D2F859
S3150800167010340D4AC3F3C203032B0FD1F8BD00F093
S31508001680FFF839E70A4D5CE7012B09BF6368402379
S31508001690084AB3FBF2F308BF9BB26DE7D2F81034E1
S315080016A0C3F3C203E8E700BF004002581C0000204D
S315080016B00090D00340420F0008B509282CD8DFE86F
S315080016C000F00A051C0A0D0D10131619154B18887B
S315080016D0154B584308BD134B5888F9E7114B9888A2
S315080016E0F6E7104BD888F3E70E4B1889F0E70D4B51
S315080016F05889EDE70B4B9889EAE70C4BD3F84C343D
S3150800170013F0405FC3F3017208D0022A08D1054BD3
S31508001710188C4FF47A73DCE700F0A8F80448D9E788
S315080017200020D7E71C00002040420F000040025866
S315080017300090D0034309012200F01F0003F1B043D3
S31508001740824003F5113319680A431A607047FEE7A9
S315080017507047000038B51D4A1D4B1E498B4220D3E1
S315080017601D4A0021934221D34FF0E0231B4C1C4D08
S31508001770D3F8142D42F40072C3F8142DD3F8882D2B
S3150800178042F47002C3F8882DAC4212D3154C164D9C
S31508001790AC4212D3154CFEF7AFFD154DAC4210D333
S315080017A038BD52F8040B43F8040BD7E743F8041B7B
S315080017B0D8E754F8043B9847E6E754F8043B9847BB
S315080017C0E6E754F8043B9847E8E700BF3C1B0008E7
S315080017D000000020400000206C0000203C1B000890
S315080017E03C1B00083C1B00083C1B00083C1B00086F
S315080017F03C1B000820F07F404FF0E02358617047FB
S315080018004FF0E02200F00400136923F004030343B9
S31508001810136170474FF0E022136943F00203136126
S3150800182070474FF0E022136943F0010313617047D4
S315080018304FF0E02300229A61704740F0BF604FF0F6
S31508001840E02340F40030C3F80C0D7047952804D9FE
S3150800185000F00F00044BC154704700F1604000F5DA
S3150800186064400170704700BF14ED00E0FEE7000019
S31508001870024A136843F480731360704700200052CD
S31508001880024A136823F480731360704700200052DD
S31508001890034A136823F00F0303431360704700BF1E
S315080018A000200052044AD2F80C3823F0070343F00C
S315080018B00203C2F80C38704700400258044AD2F8AE
S315080018C00C3823F0070343F00603C2F80C387047B8
S315080018D00040025808B50B0170B943F004030948E3
S315080018E05242D0F80C1802F0020221F03F010A43D6
S315080018F01A43C0F80C2808BD09B9FFF7B7FF43F02B
S315080019000C03ECE700400258044AD2F80C3823F0DE
S31508001910070343F00103C2F80C3870470040025829
S31508001920044AD2F80C3823F0070343F00503C2F83B
S315080019300C3870470040025808B5072807D8DFE872
S3150800194000F0040C0F12121D1D21FFF7B7FF0F4AF6
S31508001950D2F804389B04FBD508BDFFF7E1FFF6E78C
S31508001960FFF7A0FFF3E7A0F1040C0021DCF1000269
S3150800197042EB0C020020FFF7ADFFE8E705384242CC
S315080019804241F7E7FFF7C0FFE1E700BF0040025812
S31508001990F8B5074608B9FFF769FF204B421E204EE7
S315080019A01B68C3F30B03B3F5906F0FD1D6F818383D
S315080019B01C4923F440438A5C43EA8233C6F8183844
S315080019C0174AD2F818389B04FBD5F8BD1649B3F563
S315080019D08A6FD6F818588C5C25F440454FEA84344B
S315080019E018D141F68160FFF7A5FE012F4FF0B043ED
S315080019F00AD145F44045C6F81858D3F82C2442F0C5
S31508001A000102C3F82C24DBE7D3F82C2422F00102C8
S31508001A10C3F82C242C43C6F81848D1E70010005CFC
S31508001A2000400258361B0008321B0008032A30B44F
S31508001A3012D941EA0004A40784460B4621D1194667
S31508001A40604653F8044B5CF8045BA54219D1043A86
S31508001A50032AF4D860461946541E7AB1431E013942
S31508001A60021901E09A4209D013F8010F11F801CFC3
S31508001A706045F7D0A0EB0C0030BC7047002030BCA6
S31508001A807047541EEAE700BF830730B546D084186E
S31508001A90844604E003F8011B9D0704D09C46A44530
S31508001AA06346F7D130BD013A0244A2EB0C02032A81
S31508001AB029D9CCB204EB04240F2A04EB04442FD909
S31508001AC0A2F1100C2CF00F0C03F11005AC44C3E97D
S31508001AD00044C3E9024410336345F8D112F00C0FF1
S31508001AE002F00F0E18D02EF0030C9C44AEF104053C
S31508001AF01A4642F8044B6245FBD125F00304043329
S31508001B000EF003022344002ACCD0C9B21A4403F8C3
S31508001B10011B9342FBD130BD7246F4E70346C6E784
S31508001B209646E0E71400140014002C01C800F401DE
S31108001B300A000003020103020100000085
S31508001B3C0000000F0000000000000000000000007C
S31508001B4C0000000000000000241B000840004000B4
S31508001B5C400040004000400040000000000000002B
S31508001B6C000000000000000000000000000000005B
S7050800175586
